:10000000830102308A00A42AFC0003088301D8007F
:100010000408D9000A08DA008A017008DF007108B4
:10002000E0007208E1007308E2007408E30075085C
:10003000E4007608E5007708E6007808E70079082C
:10004000E8007A08E9007B08EA006C08EB005D082C
:10005000DB005E08DC0083120B1C432A0317060832
:10006000B8003706B90097080319391EE228DF01E6
:10007000151C3C281030DF00BA0111083A020318A1
:100080007F281308BB00060810395F06031D53289C
:10009000BB0B4B283F2A000000004328BB0B512814
:1000A0003F2A00000000060810395F06031D4E2895
:1000B000951A60283A08433E84008317060874287E
:1000C0000608BC000608BD000608BE003A08433E0C
:1000D000840083173C083E05F0003D083E05F10012
:1000E0003C083D05710470048000151D7C280A162B
:1000F0008A1181240A128A110317BA0A3D28951C15
:10010000A3281408BB00060810395F06031D9328B6
:10011000BB0B8B283F2A000000008328BB0B9128D3
:100120003F2A00000000060810395F0603199E28C8
:100130008E28BB0B9C283F2A0000000006081039BF
:100140005F060319992899019A019B019C01C31C20
:100150001914C41C9914C51C1915C61C9915C71C63
:100160001916C81C9916C91C1917CA1C9917CB1C3B
:100170001A14CC1C9A14CD1C1A15CE1C9A15CF1C1F
:100180001A16D01C9A16D11C1A17D21C9A17D31CF7
:100190001B14D41C9B14D51C1B15D61C9B15D71CDB
:1001A0001B16D81C9B16D91C1B17DA1C9B17DB1CB3
:1001B0001C14DC1C9C14DD1C1C15DE1C9C159701FA
:1001C000970A3F2AA4080319B91E9129DF01221CAE
:1001D000EB282030DF00BA011E083A0203182E294E
:1001E0002008BB00060820395F06031D0229BB0B4F
:1001F000FA283F2A00000000F228BB0B00293F2A02
:1002000000000000060820395F06031DFD28A21A21
:100210000F293A08433E840083170608232906085D
:10022000BC000608BD000608BE003A08433E840034
:1002300083173C083E05F0003D083E05F1003C08F0
:100240003D05710470048000221D2B290A168A11B5
:1002500081240A128A110317BA0AEC28A21C522917
:100260002108BB00060820395F06031D4229BB0B8D
:100270003A293F2A000000003229BB0B40293F2ABF
:1002800000000000060820395F0603194D293D29AA
:10029000BB0B4B293F2A00000000060820395F06EF
:1002A00003194829A601A701A801A901431D261485
:1002B000441DA614451D2615461DA615471D2616C8
:1002C000481DA616491D26174A1DA6174B1D2714A3
:1002D0004C1DA7144D1D27154E1DA7154F1D271684
:1002E000501DA716511D2717521DA717531D28145F
:1002F000541DA814551D2815561DA815571D281640
:10030000581DA816591D28175A1DA8175B1D29141A
:100310005C1DA9145D1D29155E1DA915A401A40A63
:100320003F2AB1080319391F3F2ADF012F1C9A29E0
:100330004030DF00BA012B083A020318DD292D08EE
:10034000BB00060840395F06031DB129BB0BA92974
:100350003F2A00000000A129BB0BAF293F2A000063
:100360000000060840395F06031DAC29AF1ABE29FC
:100370003A08433E840083170608D2290608BC00C9
:100380000608BD000608BE003A08433E84008317F5
:100390003C083E05F0003D083E05F1003C083D05E7
:1003A0007104700480002F1DDA290A168A11812435
:1003B0000A128A110317BA0A9B29AF1C012A2E08B8
:1003C000BB00060840395F06031DF129BB0BE92974
:1003D0003F2A00000000E129BB0BEF293F2A000063
:1003E0000000060840395F060319FC29EC29BB0B05
:1003F000FA293F2A00000000060840395F06031969
:10040000F729B301B401B501B601C31D3314C41DEE
:10041000B314C51D3315C61DB315C71D3316C81D2E
:10042000B316C91D3317CA1DB317CB1D3414CC1D09
:10043000B414CD1D3415CE1DB415CF1D3416D01DEA
:10044000B416D11D3417D21DB417D31D3514D41DC5
:10045000B514D51D3515D61DB515D71D3516D81DA6
:10046000B516D91D3517DA1DB517DB1D3614DC1D81
:10047000B614DD1D3615DE1DB615B101B10A06082C
:10048000B7000B10831203130C1D672A8316201567
:100490004308C7004408C8004508C9004608CA0008
:1004A000831215088316C300831216088316C4002E
:1004B0004108C5004208C60083120C1C662A831638
:1004C000C41B652AC50A0319C60A83120C110A1631
:1004D0008A1181240A128A118316201F7B2A073071
:1004E000D1000A168A1534240A168A1577250A12AD
:1004F0008A1183162013031383125F08F00060082B
:10050000F1006108F2006208F3006308F400640877
:10051000F5006508F6006608F7006708F800680847
:10052000F9006908FA006A08FB006B08EC005B0838
:10053000DD005C08DE00590884005A088A0058086B
:100540008300FC0E7C0E0900203084005830BD2250
:10055000A0308400D330BD22103084006030831777
:10056000BD2290308400F0308317BD2283010A162B
:100570008A11E12804068001840A04060319003464
:10058000BA2ADD00DE1BCD2A5E1BD52A5E088A0052
:100590005D08DD0A0319DE0A820083135E188317E3
:1005A0005D08DD0A840000080800831203135E0C56
:1005B0001F3903178F0003135D0C03178D0083167B
:1005C0008C170C140000000083120C0803135D1834
:1005D000F02A031703108C1B03140E0D8312031350
:1005E0007F3908006E346E3469346C346C340034F6
:1005F000723435342034623431340034643472342B
:100600006F343334353430340034F5306136793971
:100610006F00F0392036803C34196931003AE637F2
:100620007333F4327300EC32E332003AEE34653A5D
:100630007337740072347000EC37701080376F3786
:100640006400F23466108037EE376F00F0392036E0
:1006500000376F3AEC376100F43AE637003369321D
:10066000203965397000EC376E1080328031693284
:100670008030AD18801C2D18801C63313732620029
:10068000EE34001B733465346C3465346334743475
:100690000034633465346E34743465347234003439
:1006A0000A128A15AA2F0A128A1500280A128A1518
:1006B0007E2D0A128A15592D0A128A15022D0A1644
:1006C0008A15B22B0A128A15F22D0A128A15782F72
:1006D0000A128A15B52D0A168A15922B0A128A1546
:0206E0004C2F9D
:1006E40083120313C600903A031D7A2B1730812B13
:1006F400B0304606031D802B1B30812B1F30C700F2
:100704004608043E840083170008F000840A0008A9
:10071400F100840A0008F200840A0008F30070085B
:100724008316B6007108B7007208B8007308B900E0
:10073400831247088316BE000A128A11CF2BA32BFB
:100744006400831603178C18A22B03133E0883122C
:1007540003178D00831603133F08831203178C00BD
:1007640083168C1303108B1B03148B130C15553039
:100774008D00AA308D008C140C1103188B170313F1
:1007840083120800831603133608BF00A1238316BF
:10079400BE0A3708BF00A12B831603133608BF0017
:1007A400A1238316BE0A3708BF00A1238316BE0AFD
:1007B4003808BF00A1238316BE0A3908BF00A12B45
:1007C400831203133A08073A031D0800672E031720
:1007D4002818F22B413083120313C1004630F72B43
:1007E4005E3083120313C1004630C20090300A12F7
:0C07F4008A1503200A128A1183160317CD
:100800004818082C413083120313C10046300D2CC8
:100810005E3083120313C1004630C200B0300A12AA
:100820008A1503200A128A118316031768181E2CD2
:10083000413083120313C1004630702D5E308312A5
:100840000313C1004630702D0317A8182D2C373024
:1008500083120313C1004630322C65308312031318
:10086000C1004630C20090300A128A1503200A12D5
:100870008A1183160317C818432C373083120313C9
:10088000C1004630482C653083120313C100463046
:10089000C200B0300A128A1503200A128A11831688
:1008A0000317E818592C373083120313C100463060
:1008B000702D653083120313C1004630702D8312F2
:1008C00003171008023A031D6A2C7A300313C10083
:1008D0004630752C100B712C7F300313C10046304D
:1008E000752C18300313C1004630C20090300A1234
:1008F0008A1503200A128A1103171D08023A031DE4
:10090000862C7A300313C1004630912C1D0B8D2CA0
:100910007F300313C1004630912C18300313C100FF
:100920004630C200B0300A128A1503200A128A111A
:1009300003172A08023A031DA22C7A300313C100C0
:100940004630702D2A0BA92C7F300313C10046308E
:10095000702D18300313C1004630702D6C30831297
:10096000C1004630C20090300A128A1503200A30B6
:10097000F200F301831603172608F1002508F000A2
:100980000A168A154924740883120313C1007508D6
:10099000C20090300A168A15B9256C30C100463065
:1009A000C200B0300A128A1503200A30F200F301A7
:1009B000831603174608F1004508F0000A168A1549
:1009C0004924740883120313C1007508C200B030B3
:1009D0000A168A15B9256C30C1004630C200D030E5
:1009E0000A128A1503200A30F200F3018316031756
:1009F0006608F1006508F0000A168A1549240A12F3
:100A00008A11740883120313C1007508C200402DB7
:100A100033308312C1004630C20090300A128A156A
:100A2000032083160317270883120313C100C20192
:100A300090300A168A15B9253330C1004630C200FD
:100A4000B0300A128A150320831603174708831251
:100A50000313C100C201B0300A168A15B92533301C
:100A6000C1004630C200D0300A128A1503200A1293
:100A70008A1183160317670883120313C100C2018A
:100A8000D030D82D83120317951A4B2D4B300313FA
:100A9000C10046304F2D11300313C1004630C20053
:100AA00090300A128A1503200A128A110317A21A1B
:100AB0005E2D4B300313C1004630622D11300313FD
:100AC000C1004630C200B0300A128A1503200A1253
:100AD0008A110317AF1A732D4B300313C100463030
:100AE000C200D030CD2D11300313C1004630702D1F
:100AF0002C308312C1004630C20090300A128A1591
:100B00000320B0300A168A151F2483164F0883125B
:100B1000C100C201B0300A168A15B9250A128A111D
:100B2000AD2D0A308312C1004630C20090300A1247
:100B30008A1503200A128A118316211CA42D48301D
:100B40008312C1004630A82D5A308312C1004630AE
:100B5000C200B0300A128A150320D0300A168A1556
:100B60001F240A128A11892E57308312C100463081
:100B7000C20090300A128A150320B0300A168A1576
:100B80001F240A128A118316B508031DD32D3E3087
:100B90008312C1004630C200B0300A128A15032009
:100BA0000A128A11892E35088312C100C201B030A1
:100BB0000A168A15B9250A128A11892EBE01053036
:100BC000BF00A1238316BE01BE0A03172708031323
:100BD000BF00A12302308316BE000317470803138A
:100BE000BF00A12303308316BE0003176708031359
:100BF000BF00A12390308B260A128A11B0308B26B9
:100C00000A128A11D0308B260A128A1107308316F5
:100C1000BE0083120317100883160313BF00A1231D
:100C200008308316BE00831203171D0883160313B2
:100C3000BF00A12309308316BE00831203172A08C0
:100C400083160313BF00A12383160317250803137C
:100C5000B600031726080313B7000A30BE00C423EA
:100C60000A128A118316031745080313B6000317E7
:100C700046080313B7000C30BE00C4230A128A11C1
:100C80008316031765080313B600031766080313DA
:100C9000B7000E30BE00C4230A128A11103083162A
:100CA000BE004F08BF00A12311308316BE002108EB
:100CB0000139BF00A12312308316BE003508BF00E2
:100CC000A1230A128A15D2240A128A11892E8316A8
:100CD00023080319612E013A0319E92B033A03197A
:100CE000242C013A03195F2C073A0319AE2C013A60
:100CF0000319082D033A0319422D013A0319782DDF
:100D00000F3A0319912D013A0319B42D033A03192F
:100D1000DE2D8312080083120313C200903A031DD4
:100D2000952E0430C1001030A02EB0304206031DB5
:100D30009D2E0530C1001D30A02E0630C1002A3086
:100D4000C3008316B60183124208183E840083173D
:100D500083160018361483124308053E8400831757
:100D60008316801AB61483124208183E8400831733
:100D7000831680183615831241088316BE00360884
:100D8000BF00A12B83160313B60120183614A01937
:100D9000B614201A36151330BE003608BF00A12B3A
:100DA000F601F401F50172087304031900341F30D1
:100DB000F6040310F60AF20DF30D031CDA2EF30C01
:100DC000F20C73087102031DE72E72087002031CF7
:100DD000EF2E7208F0027308031C730AF102F40D7F
:100DE000F50DF60BF61ADF2EF61FFB2EF409F40AAA
:100DF0000319F503F5097408F2007508F300761F6E
:100E00000034F009F00A0319F103F1090034000875
:100E1000F000840A0008F100840A0008F200840A45
:100E20000008F300142F840183120313EC01F31F55
:100E3000282F0310FF30F007F009031CF107F10918
:100E4000031CF207F209031CF307F3096C17EC17F4
:100E500077088039EC06F71F3F2F0310FF30F407A7
:100E6000F409031CF507F509031CF607F609031C32
:100E7000F707F7093F2F840183120313EC01F801F0
:100E8000F901FA01FB01740875047604770403196B
:100E90004C2FC030EC05572FF001F101F201F301A6
:100EA000F12F0310F40DF50DF60DF70DEC0AF71FF9
:100EB000512FEC0A0310F80DF90DFA0DFB0D770810
:100EC0007302031D6D2F76087202031D6D2F7508C6
:100ED0007102031D6D2F74087002031C7F2F78149C
:100EE0007408F0027508031C750FF1027608031CE4
:100EF000760FF2027708031C770FF3020310F70C4A
:100F0000F60CF50CF40CEC036C083F39031D5A2F5A
:100F10006C1F972F0310FF30F007F009031CF10737
:100F2000F109031CF207F209031CF307F309700827
:100F3000F4007108F5007208F6007308F7007808ED
:100F4000F0007908F1007A08F2007B08F300EC1F4A
:100F5000F12F0310FF30F007F009031CF107F1092E
:100F6000031CF207F209031CF307F309F12F8401B4
:100F70007008F8007108F9007208FA007308FB00A5
:100F8000F201F301F001F1010310FB0CFA0CF90C72
:100F9000F80C031CD92F7408F00775080318750F97
:100FA000F10776080318760FF20777080318770F12
:100FB000F307780879047A047B040319F12F0310EE
:100FC000F40DF50DF60DF70DC42F0008F000840A9E
:100FD0000008F100840A0008F200840A0008F30007
:100FE000B82F840803190034730880008403720842
:100FF000800084037108800084037008800000343E
:1010000003138312080083120313C3001F3E8400DE
:101010008317023080000630C700C801C7034808A4
:101020004107DD004208DE005D080318DE0A0A12EF
:101030008A11C1220A128A15C600C6080319582847
:101040004608203A031D2628C501432846082D3AA4
:10105000031D2C2840304228613046024608031CFC
:101060003A289F3EC40018308A00440833200A12F0
:101070008A154228D03EC40018308A0044084E2009
:101080000A128A15C50047084307193E84008317D2
:1010900045088000C80A06304802031858280E2860
:1010A00047084307193E840083178001C703C80A15
:1010B00006304802031808005028831203173F081F
:1010C000F0004008F1004108F2004208F300F00986
:1010D000F109F209F309F00A0319F10A0319F20AF6
:1010E0000319F30A7008BF007108C0007208C1003C
:1010F0007308C2000313080083120313BD00031713
:10110000C11F8428FF30C20403133D08183E840029
:101110008317001C8C285D203D080C3E840083173B
:101120000008F000840A0008F100840A0008F200B8
:10113000840A0008F30070080317BF077108031C36
:10114000A628710A0319F20A0319F30AC0077208E4
:10115000031CAD28720A0319F30AC10773080318A8
:10116000730AC20703133D08173E840083178008E3
:1011700003199A293D08840083170008F000840AA7
:101180000008F100840A0008F200840A0008F30055
:10119000700803173F02F4004008F5007108031CB3
:1011A000710FF5024108F6007208031C720FF60277
:1011B0004208F7007308031C730FF7027408031347
:1011C000CC007508CD007608CE007708CF000A164F
:1011D0008A15A1240A128A157008BE007108BF0082
:1011E0007208C0007308C1003D08173E84008317D1
:1011F0000008F000F101F201F3017308803AF400F5
:101200004108803A7402031D0F2940087202031D31
:101210000F293F087102031D0F293E087002831237
:1012200003133D0803182429143E8400831780010A
:101230003D08103E840083178001840A8001840ADF
:101240008001840A80019A29143E840083170830A3
:1012500000023D0803188429143E84008317800A85
:101260003D08103E840083170008F000840A00083F
:10127000F100840A0008F200840A0008F300031752
:101280003F087007F4007108F50040080318400F8C
:10129000F5077208F60041080318410FF6077308B6
:1012A000F70042080318420FF70774080313BE0043
:1012B0007508BF007608C0007708C1003D08103EE1
:1012C000840083173E088000840A3F088000840A57
:1012D00040088000840A410880003D08143E8400D4
:1012E00083170008083A031D9A293E08F0003F08BA
:1012F000F1004008F2004108F30003300A168A1595
:10130000A7230A128A159129840083170008F00088
:10131000840A0008F100840A0008F200840A000828
:10132000F30070080317BF007108C0007208C10005
:101330007308C20003133D088400831703173F0896
:101340008000840A40088000840A41088000840AE2
:101350004208800083160313A01CB22983123D08A3
:10136000083EB52983123D08043E84008317000817
:10137000F000840A0008F100840A0008F200840AE0
:101380000008F30070080317BF0271080318CD2985
:10139000710A0319F20A0319F30AC002720803184A
:1013A000D429720A0319F30AC1027308031C730AD1
:1013B000C20203133D08183E84008317801C0800F6
:1013C0005D2883120313BD00093E840083170008C3
:1013D000F000840A0008F100840A0008F200840A80
:1013E0000008F3007008BE007108BF007208C0005A
:1013F0007308C1003D0884008317000B172A4008BA
:10140000C2000F30C005C1013E080317BF0003131F
:101410003F080317C000031340080317C10003135C
:1014200041080317C2000313421E08004D2A3D085D
:10143000840083170008023A031D4F2A4108C200A6
:1014400040080F39A5003F0E0F39A7003F080F399C
:10145000A3003E0E0F39A6003E080F39A4000A165D
:101460008A15D6240A128A152008BE002108BF005A
:101470002208C000C1013E080317BF0003133F0844
:101480000317C000031340080317C10003134108EA
:101490000317C2000313421C08005D205F2AC1012C
:1014A0003E080317BF0003133F080317C0000313D0
:1014B00040080317C100031341080317C2000313B8
:1014C00008008B13831603133308B1003408B200ED
:1014D000A0128B17831208003C30F2000230F30098
:1014E000831603133508F000F1010A168A15492402
:1014F0000A128A157408B3007508B400612A8316AD
:101500000313AE08031D9B2A03179C019D019E0136
:101510009F01BC01BD01BE01BF01DC01DD01DE0197
:10152000DF010313A601A701A801A901AA01AB01CC
:10153000AC01AD01192B2E08BE00BE030310BE0D79
:101540000310BE0D0310BE0D2C30BE073E087223E3
:101550008316360837083808390836088312CB0056
:10156000831637088312CC00831638088312CD0007
:10157000831639088312CE0090300A168A158E27FA
:1015800070088316A6007108A7007208A8007308E7
:10159000A900290DA90CA80CA70CA60C36088312CB
:1015A000CB00831637088312CC00831638088312C9
:1015B000CD00831639088312CE00B0300A168A1582
:1015C0008E270A128A1570088316AA007108AB00CC
:1015D0007208AC007308AD002D0DAD0CAC0CAB0C5B
:1015E000AA0C3E0ABE007223831636083708380854
:1015F000390836088312CB00831637088312CC00D3
:10160000831638088312CD00831639088312CE0062
:10161000D0300A168A158E270A128A15700883168A
:101620000317DC007108DD007208DE007308DF00BC
:101630000313831208004A2B0A128A15D2240A12B5
:101640008A15552B25308312C1004630C2009030D8
:101650000A128A1503205230C1004630C200B03051
:101660000A128A1503207630C1004630C200D030FD
:101670000A128A1503200A128A15552B7F2214306C
:101680008316BE002E08BF000A128A11A1230A1277
:101690008A151C2B83160313230803191C2B013AEC
:1016A0000319222B033A03193E2B831208008316D9
:1016B00003133E08831203178D0083168C130C143A
:1016C00083120C0883160313BF00831208005723EC
:1016D00083163F08B600BE0A572383163F08B7009B
:1016E00083120800572383163F08B600BE0A57230B
:1016F00083163F08B700BE0A572383163F08B80079
:10170000BE0A572383163F08B900831208008316C8
:101710000313BE01572383163F08053A031D742C9B
:10172000BE01BE0A572383163F080317A7000430E3
:101730000313BE00572383163F08B6000317281073
:101740000313361CA52B03172814831203179512B5
:1017500083160313B61CB02B83120317951683163A
:101760000317A8100313361DB72B0317A814023054
:101770000313BE00572383163F080317C700053025
:101780000313BE00572383163F08B6000317481003
:101790000313361CCD2B0317481483120317A21210
:1017A00083160313B61CD82B83120317A2168316B5
:1017B0000317C8100313361DDF2B0317C81403309B
:1017C0000313BE00572383163F080317E7000630B4
:1017D0000313BE00572383163F08B6000317681093
:1017E0000313361CF52B0317681483120317AF126B
:1017F00083160313B61C002C83120317AF1683162F
:101800000317E8100313361D072C0317E8140730DD
:101810000313BE00572383163F088312031790005B
:1018200010300A168A1145230A128A1508308316C9
:10183000BE00572383163F08831203179D001D30F7
:101840000A168A1145230A128A1509308316BE002A
:10185000572383163F0883120317AA002A300A165B
:101860008A1145230A128A150A308316BE0067239F
:101870000A128A15831636080317A50003133708C2
:101880000317A6000C300313BE0067230A128A1543
:10189000831636080317C500031337080317C6005D
:1018A0000E300313BE0067230A128A15831636080A
:1018B0000317E500031337080317E600103003137E
:1018C000BE00572383163F08CF001130BE005723B8
:1018D000831621083F06FE393F06A1001230BE00E4
:1018E000572383163F08B5001730BE0072230A1233
:1018F0008A15831636080317940003133708031755
:1019000095000313380803179600031339080317CB
:1019100097001B300313BE0072230A128A15831628
:1019200036080317B400031337080317B500031371
:1019300038080317B600031339080317B7001F3020
:101940000313BE0072230A128A1583163608031782
:10195000D400031337080317D500031338080317FF
:10196000D600031339080317D70013300313BE0042
:10197000572383163F08B600361CC02C2014D214FF
:10198000B618A015361920161430BE00572383163A
:101990003F08B600AE007F220A128A1596308316E1
:1019A000AF006C2A83160317AF080319E02C9030A0
:1019B0000A168A151F240A128A1583160317AF0107
:1019C000CF080319EC2CB0300A168A151F240A120E
:1019D0008A1583160317CF01EF080319F82CD030AE
:1019E0000A168A151F240A128A1583160317EF0197
:1019F000E3300313D20507308312BA008316A20125
:101A000083120800831603132208023A031D122DC5
:101A100024080A168A112D220A128A15D2240A12C3
:101A20008A15572D2208033A031D1D2D24080A1676
:101A30008A15FD250A128A150E2D2208053A031D66
:101A4000422D83123A08073A831603193B2D2308C7
:101A5000043A031D312D0A168A1500250A128A152B
:101A60003C2D2308053A031D3C2D0A168A157424C3
:101A70000A128A153C2DA30A0A128A11E2230A12BD
:101A80008A15572D2208073A031D4D2DA30A0A1661
:101A90008A11DD230A128A15572D2208083A031DE0
:101AA000572DA30A0A128A151B230A128A158312BC
:101AB0000800831203133A08073A031D692D8316A1
:101AC0002208053A031D682DA3030A128A11E22B8E
:101AD000D32C3A083806031D742D0730B80083163E
:101AE00024080A168A114A28BA08031D782DD22C18
:101AF000BA03831624080A168A114A28831203138C
:101B0000AF08031D852D90308C2D2F08023A031D40
:101B10008B2DB0308C2DD030BD0083162208023AB8
:101B2000031D9C2D240883123D06031D9B2D3A089E
:101B3000073A0319A22D8316A208031DB32DA01C7A
:101B4000AC2D83123D080A168A112D220A128A151D
:101B5000D2240A128A15B32D0230A2005215831224
:101B60003D088316A4008312080083160313A208FD
:101B7000031DC42D0130A0060230D2060A128A11BC
:101B8000C2260A128A15CD2D2208043A031DCD2D36
:101B90008030A006D2240A128A158312080083120C
:101BA0000313C4000A168A151F24BA01B91007309E
:101BB000B8004108BB004208BC003911C308031D2E
:101BC000391544081F3E840083178001800A83165C
:101BD000D215831244088316A400831244080A16FF
:101BE0008A114A28831203132F08043A031DFA2D81
:101BF000BE01022E2F08033CBE0003103E0DBE079F
:101C00002E03BE0783162208023A8312031D212EDB
:101C10003A08073A031D212E8316201C142E033088
:101C20008312C1000230182E02308312C10003302B
:101C3000C200C301C30A83162408CF250A128A15DD
:101C400083123A08073A0319492E3808073A031D48
:101C5000342E3B083A020318492FBA08031D3A2EC6
:101C6000BE080319492F3A2E3C083807BD003A0236
:101C70000318492FBA0A3A03323E840083133E0800
:101C80008000831624080A168A114A200A128A152F
:101C9000492F83162208043A0319A42EBB2E0530BF
:101CA0008316A200A301A30A0A128A11E2230A12D0
:101CB0008A15492F06308316A20049308312C100CD
:101CC0000330C20090300A128A1503204230C1004E
:101CD0000330C200B0300A128A150320D0300A1631
:101CE0008A151F240A128A15492F07308316A2006D
:101CF000A301A30A0A168A11DD230A128A15492FA5
:101D000008308316A200A301A30A0A128A151B2316
:101D10000A128A15492F8316211C962E0830A00618
:101D200020120A128A11C2260A128A15D2240A1215
:101D30008A15492F8316211C962E1030A006A0115B
:101D4000912E8316A016962E83123E0803194F2E4D
:101D5000013A03195A2E043A0319752E033A03194E
:101D6000802E013A03198B2E0F3A03199A2E013A4D
:101D70000319A12E962E2208073A031DC72E83129F
:101D8000BE080319492F3E088316AE00792E22089B
:101D9000083A031DD02E83123E088316AE00842E0F
:101DA000A208031D492F03179C019D019E019F015D
:101DB000BC01BD01BE01BF01392F83162A08F00006
:101DC0002B08F1002C08F2002D08F300F009F109AE
:101DD000F209F309F00A0319F10A0319F20A0319C7
:101DE000F30A70080317BC007108BD007208BE003A
:101DF0007308BF00492F83162608F0002708F1005A
:101E00002808F2002908F300F009F109F209F309A2
:101E1000F00A0319F10A0319F20A0319F30A700808
:101E200003179C0071089D0072089E0073089F00B4
:101E3000492F8316260803179C000313270803174E
:101E40009D000313280803179E0003132908031796
:101E5000172F83162A080317BC0003132B08031738
:101E6000BD0003132C080317BE0003132D0803172E
:101E7000F92E831203133E08023A0319DD2E063AA7
:101E80000319FB2E023A0319192F0E3A031D0800FD
:101E9000292F031383120800831603132208023A22
:101EA0008312031D6C2F3A08073A031D6C2F83160B
:101EB000201C5F2F03308312C1000230632F0230D9
:101EC0008312C1000330C200C301C30A8316240871
:101ED000CF250A128A1583123A08073A031D391DC5
:101EE00008000230B906831624080A168A114A2807
:101EF000831603132208023A8312031D982F3A080F
:101F0000073A031D982F8316201C8B2F0330831252
:101F1000C10002308F2F02308312C1000330C20093
:101F2000C301C30A83162408CF250A128A15831217
:101F30003A08073A031908003808073A031D080051
:101F4000BC08031908003A08B800831624080A16CA
:101F50008A114A2883120313AF08031DB42F90304F
:101F60008316A4001030BC2F2F08023A031DBE2F89
:101F7000B0308316A4001D30A500F22FD030831698
:101F8000A4002A30BC2F0330A200201CD42F033021
:101F90008312C1000230C200C301C30A83162408A1
:101FA000CF250A128A15FE2F02308312C10003309A
:101FB000CB2F0A168A15B9240A128A15D2240A12BE
:101FC0008A15FE2F0A168A1132210A128A11E2237B
:101FD0000A128A15FE2F24080A168A15AD260A123F
:101FE0008A15DE2F22080319C32F043A0319D92FAB
:101FF000013A0319E22F033A0319EB2F8312080069
:10200000831203138701F830831687048312851423
:1020100005110710871005100430D7000708D600F7
:10202000D70B0E280708A900851005150430D70026
:102030000708D600D70B18280708AA0005110714AF
:102040000430D7000708D600D70B22280708AB00BA
:10205000071087140430D7000708D600D70B2C28A8
:102060000708AC00871005140430D7000708D60015
:10207000D70B36280708AD00073083168705831273
:10208000051087018514051586178510051186131F
:102090003914080083120313C8001F3E84008317FD
:1020A000000B0800BA08031D61284808193E840087
:1020B00083170A168A154F200A168A118000C90153
:1020C00085283A08C700C9013A0849060319862835
:1020D000C7034708323E840083130008C500183048
:1020E0008A0045084E200A168A11C600490848078A
:1020F000193E8400831746088000C90A64284908ED
:102100004807193E840083178001C90A0630490236
:10211000031C7F283808073A0319A52838083A0213
:10212000C900B808031D9F2849084807193E8400C4
:1021300083170A168A154F200A168A11800049084B
:102140004807193E840083178017B91C0800B80897
:10215000031DBA08031DB4283A0848071A3E840034
:1021600083174030800008003A084807193E840071
:102170008317403080000800383083120313850035
:10218000831685010130831286007E308316860017
:1021900083128701043083168700D43081003130E8
:1021A000831290000630920094308316920007301C
:1021B0008C0068308B0006309F000430831297003B
:1021C0000800BC2010300A168A11CB231D300A16D5
:1021D0008A11CB232A300A168A11CB231030BD0076
:1021E00090300A168A158A241D30BD00B0300A16B8
:1021F0008A158A242A30BD00D0300A168A158A240E
:102200000A168A158C230A168A1587230A128A153C
:102210008723FE30C1000230C20090300A128A15B6
:102220000320F830C1000230C200B0300A128A1513
:102230000320F230C1000230C200D0300A128A15E9
:1022400003208316A201A20A8B170A168A151D27DE
:102250000A168A11B5220A168A11DA250A168A1177
:10226000640025298C292408183E84008317013036
:102270008006A8292408183E8400831702303829D4
:10228000250884008317800A250884008317000826
:10229000033A031D4F292508840083178001250870
:1022A0000A168A1145230A168A11A82905308312B5
:1022B000C100C201C301831624080A128A15CF2562
:1022C0000A168A11A829023057292508053E8400DC
:1022D000831720303829CF0BA8290530CF00A82933
:1022E0000130A106A829B508031D78290F308329DC
:1022F00035080F3A031D7E291E30832935081E3A02
:10230000031D85293C30B5008629B5010A128A15BE
:102310006C220A168A11A829831603132308F000D9
:102320000130F002031CA829093070020318A82903
:1023300011308A009F30700703188A0A82003329FF
:102340003A2940295629632965296B29702973295F
:102350008312080083120313D0002030F4000330EE
:10236000F500F601F7014C08F0004D08F1004E08A9
:10237000F2004F08F3000A128A11B7270A168A11D1
:102380007008D1007108D2007208D3007308D4001D
:102390005008153E840083170008F000840A0008E6
:1023A000F1000310F10CF00C7008D500D41FDA29ED
:1023B000D509D50A5508D10701300318D2070318EB
:1023C000D3070318D4075008153E8400831700086C
:1023D000F000840A0008F1007008F4007108F500AC
:1023E000F601F7015130840083130A128A1107277E
:1023F0000A168A1183160313201C222A7F30F40048
:10240000F501F601F70183125130840083130A129B
:102410008A11E527193083120313D10701300318FD
:10242000D2070318D3070318D4073230F400F5019C
:10243000F601F7015130840083130A128A1107272D
:102440000A168A11831203135108F0005208F10092
:102450005308F2005408F300080083120313C1006C
:102460003A08073A031D722A4108840083170008BE
:10247000F000840A0008F100840A0008F200840ACF
:102480000008F3007008C2007108C3007208C4009D
:102490007308C5008316A01C5E2A83124108083EFB
:1024A0008400831742088000840A43088000840A5D
:1024B00044088000840A450880000800831241080F
:1024C000043E8400831742088000840A4308800089
:1024D000840A44088000840A4508800041080A12E2
:1024E0008A11722B41080A168A118E250A168A1142
:1024F0007008C2007108C3007208C4007308C500E8
:102500004108043E840083170008F000840A000894
:10251000F100840A0008F200840A0008F300700841
:10252000C2077108031C992A710A0319F20A0319D8
:10253000F30AC3077208031CA02A720A0319F30ADC
:10254000C40773080318730AC5074108043E8400D2
:10255000831742088000840A43088000840A4408E4
:102560008000840A45088000080083120313391C88
:102570000800A808031DE62AAE0105302E022E0829
:102580000318DA2A293E840083130008B100AF0142
:10259000B119D92AAF0A311AD92AAF0AB11AD92AE0
:1025A000AF0A311BD92AAF0AB11BD92AAF0AAE0A2A
:1025B000BD2A2E08053A0319432B2F08053A0319A3
:1025C000432BB001B00AA801A80A432B2E08293ECC
:1025D000840083130008B100AF08031DF12A0830FE
:1025E000022B2F0BF52A1030022B2F08023A031D65
:1025F000FB2A2030022B2F08033A031D012B403009
:10260000022B8030B105B108031D0A2BB00B432B00
:10261000A801432B280B3A2BB00A3008053A031DBA
:10262000432B8316A01E1A2B0A128A1561220A1642
:102630008A11372B0530F10083122E080A168A15ED
:10264000BD232F07F0007007F0001830DE0070087F
:10265000013E0A128A11C122F0000A128A11C22216
:10266000DE0070080A128A11C1220A168A1102308D
:10267000A800432B2808023A031D432B3008053AD3
:102680000319432BB00A3910080083120313BE004C
:1026900084008317000B722B3E0A840083171830C6
:1026A00080003E08053E8400831700103E08053E6A
:1026B0008400831780103E08033E84008317FA309D
:1026C00080003E08053E8400831700153E08053E45
:1026D0008400831780153E08023E840083179930DA
:1026E000800008003E08840083170008023A031D9A
:1026F0009F2B3E0A840083171C3080003E08053E55
:102700008400831700143E08053E84008317801060
:102710003E08033E840083171F3080003E08053EBC
:102720008400831700113E08053E84008317801142
:102730003E08023E840083171F30800008003E0AD6
:1027400084008317183080003E08053E84008317FC
:1027500000143E08053E8400831780143E08033EA3
:10276000840083171F3080003E08043E84008317D6
:102770003E3080003E08053E8400831700113E086D
:10278000053E8400831780113E08023E84008317B3
:102790001F308000080083120313BD00073E840031
:1027A000831780013D08053E8400831780163D088D
:1027B0008400831780013D08452B6E2C2530831241
:1027C000C1004630C20090300A128A1503205230F0
:1027D000C1004630C200B0300A128A1503207230A0
:1027E000C1004630C200D0300A128A1503200A16F2
:1027F0008A117F2C6E308312C1004630C2009030A7
:102800000A128A150320D0300A168A151F240A16C8
:102810008A118316201C332C03308312C10002302E
:10282000C200C301B0300A128A15CF250A168A11D8
:102830007F2C0A168A11262570088316B6007108A7
:10284000B7007208B8007308B9001E308312C100C7
:102850004630C20090300A128A1503200A168A11E7
:10286000831620180C2C02308312C1000330102C68
:10287000AE080319682C0A168A11262570088316DB
:10288000BA007108BB007208BC007308BD002E08B6
:10289000BE00BE030310BE0D0310BE0D0310BE0D1F
:1028A0002C30BE0736083708380839083E080A12A7
:1028B0008A11CE2383163A08B6003B08B7003C08BD
:1028C000B8003D08B9003E0ABE000A128A11CE23A4
:1028D0000A128A15D2240A168A117F2C8316031332
:1028E00023080319682C013A0319DE2B033A031954
:1028F000FA2B013A0319192C073A0319382C8312C1
:10290000080083120B1D9C2C03171708023A031DA5
:102910008C2C960B8C2C97012408023A031D932CC7
:10292000A30B932CA4013108023A031D9A2CB00B7F
:102930009A2CB1010B11831203130C1CE02C83168B
:10294000C10A0319C20AAF080319B82CAF0BB82C7F
:102950000730D1000A168A1534240A168A15C923AD
:102960000A168A1577250A168A110A308316B000CE
:10297000320831040319C42CFF30B107031CB20321
:10298000320831040319A016B0080319DB2CB00B70
:10299000DB2C83120317980803191516A5080319D1
:1029A0002216B20803192F169801A501B2010A30A8
:1029B00083160313B000C008031DC00383120C105C
:1029C0008C1C08008316D00A4F085002031CED2C03
:1029D0000A168A159C230A168A110530831650029E
:1029E000031C232D07305102031C032D83123918B9
:1029F000012D0A168A1534240A168A1100200A1697
:102A00008A118316D101A01A212D0A168A153424A1
:102A10000A168A1106308316510203181B2D0A1656
:102A20008A15FB230A168A15EA230A168A15D92362
:102A30000A168A11202D0A168A155E240A168A1192
:102A40008316D001D10A83128C100800831203135D
:102A50003C08053CCD003808073A0319332D3808E7
:102A6000CD023A08CD070630CC004C084D020318C1
:102A7000402DCC034C08323E840083138001352D59
:102A80003A08CC00CC0803195A2DCC03CD034C08CE
:102A9000323E840083130008CB004D08323E840090
:102AA00083134B088000422DCD034D08323E840035
:102AB00083138001CD08031D542D3208A50033086F
:102AC000A7003408A3003508A6003608A4000A169B
:102AD0008A15D6240A168A112008CE002108CF00B4
:102AE0002208D000D1010730BA008316D211831218
:102AF0004E08F0004F08F1005008F2005108F300B2
:102B0000B91C0800F009F109F209F309F00A0319E8
:102B1000F10A0319F20A0319F30A080083120313D6
:102B2000C60026257008C7007108C8007208C900D1
:102B30007308CA004708CB004808CC004908CD00FC
:102B40004A08CE0046080A168A158E270A168A11E8
:102B50007008C7007108C8007208C9007308CA006D
:102B60004608183E840083174708F0004808F10023
:102B70004908F2004A08F300001C0800F009F109B6
:102B8000F209F309F00A0319F10A0319F20A031909
:102B9000F30A7008C7007108C8007208C9007308FA
:102BA000CA004708F0004808F1004908F2004A0846
:102BB000F300080083160313211CB52E2208023AE5
:102BC000031DF02D83123A08073A83160319201DBE
:102BD000F02D0A128A1502250A168A118316201171
:102BE000A019F42D201EB52EC008031DB52E0A30E5
:102BF000C000CB01CC01CD01CE01201DB02E470875
:102C00004302F0004408F1004808031C480FF10299
:102C10004508F2004908031C490FF2024608F30078
:102C20004A08031C4A0FF30270088312CC00710893
:102C3000CD007208CE007308CF000A168A15A124B1
:102C40007008BD007108BE007208BF007308C000A4
:102C50003D08F4003E08F5003F08F6004008F70084
:102C60006030F0003430F1003C30F2000230F3000C
:102C70000A128A1113270A168A1170088316CB00CC
:102C80007108CC007208CD007308CE00201EAE2E55
:102C900026088312BD00831627088312BE00831600
:102CA00028088312BF00831629088312C0006430ED
:102CB000F400F501F601F7013D30840083130A1298
:102CC0008A11E527831603172508F4002608F50066
:102CD000F601F701831203133D30840083130A12B7
:102CE0008A1107277030F400F530F500F601F7017E
:102CF000831203133D30840083130A128A11E527DF
:102D0000E030F4002E30F500F601F70183120313D2
:102D10003D30840083130A128A110727831203139C
:102D20003D08F4003E08F5003F08F6004008F700B3
:102D30008316CB30840083130A128A11E5271030E2
:102D4000F4002730F500F601F70183160313CB30AA
:102D5000840083130A128A11072783160313201194
:102D60000A168A154D260A168A1183120800831244
:102D70000313BD001F3E840083178008031D080055
:102D80008316A01F112F831203173F080313C200DD
:102D9000031740080313C300031741080313C400BB
:102DA000031742080313C5003D08193E840083172A
:102DB00018308A0042080F394E2080003D081A3E24
:102DC0008400831718308A00420E0F394E2080008D
:102DD0003D081B3E8400831718308A0043080F39D2
:102DE0004E2080003D081C3E8400831718308A0066
:102DF000430E0F394E2080003D081D3E840083178E
:102E000018308A0044080F394E2080003D081E3ECD
:102E10008400831718308A00440E0F394E2080003A
:102E20000800831203173F080313CC000317400860
:102E30000313CD00031741080313CE000317420804
:102E40000313CF000A168A15A1247008BE0071086A
:102E5000BF007208C0007308C1003E08CC003F08E4
:102E6000CD004008CE004108CF003D080A168A1167
:102E7000AA210A168A117008BE007108BF007208E4
:102E8000C0007308C1003E08C2003F08C3004008EC
:102E9000C4004108C5000330F000450DC50CC40C4A
:102EA000C30CC20CF00B4D2F4208A0004308A10038
:102EB0004408A2000A168A1537250A168A110A3014
:102EC0002502031C702F4030C6005C30C70038302C
:102ED000C8007130C9005C30CA004030CB00DB2F25
:102EE00018308A0024084E20C60018308A002608B0
:102EF0004E20C70018308A0023084E200A168A1177
:102F0000C800C901CA01CB01831620188B2F831278
:102F10003E1D8C2FC6178312A508031DAC2F8316E8
:102F2000201C9D2F8312A708031D9D2F0317C21F6E
:102F3000BE2F40300313C900BE2F18308A00831201
:102F400027084E200A168A11C9000317C21FBE2F78
:102F500040300313CA00BE2F18308A0027084E20C5
:102F6000C90018308A0025084E200A168A11CA00A6
:102F70000317C21FBE2F40300313CB008316031369
:102F8000201CC52F8312C817C72F8312C9173D08ED
:102F90000C3E840083170008F000840A0008F1004A
:102FA000840A0008F200840A0008F3007204710425
:102FB0007004031DCB173D08193E84008317460893
:102FC00080003D081A3E84008317470880003D08B2
:102FD0001B3E84008317480880003D081C3E840087
:102FE0008317490880003D081D3E840083174A0866
:102FF00080003D081E3E840083174B0880000800B7
:10300000820750340334533403345034033453347C
:1030100003345034033456340334593403345634AF
:1030200003345C340334563403345F340334623481
:103030000334623403346234033465340334683453
:10304000033462340334623403346234033462344C
:1030500003346B3403346234033462340334623433
:1030600003346E340334820777347C3439345E346D
:10307000793471343D34743404341E3400343834BB
:10308000003454345C347334003450346D34783448
:103090003E341C34003400346E345B3482073F34D9
:1030A00006345B344F3466346D347D3407347F34FA
:0E30B0006F3477347C3439345E3479347134C3
:10370E00073083120313BA00080005308316031323
:10371E00CF008312080083160313A208031D9A2BF1
:10372E000430A200521683120800831203130510F0
:10373E008701851405158617851005118613080057
:10374E00F400F40AF40303190034730DF30CF20CB5
:10375E00F10CF00CA92B83160313A208031DBB2B2F
:10376E000230A0060130D20683120800F0000030AD
:10377E00711870070310F00D0310F10CF108031906
:10378E000800BF2B973083120317180203189515E4
:10379E00973025020318A215973032020318AF1581
:1037AE0003130800831603135108E93E84008317A0
:1037BE0000088312D60005105619051487008617C7
:1037CE00861786130800831603135108C93E84001A
:1037DE00831700088312D6000510561905148700AA
:1037EE000515051505110800831603135108A93E8A
:0237FE00840045
:10380000831700088312D600051056190514870087
:10381000851485148510080083120313D7001B2C10
:103820000103D600560801060319182C6400122C57
:10383000D70383120313D70803190800102C83122F
:103840000313C5001F3E8400831702308000C601A9
:1038500046084507193E840083178001C60A0630D2
:10386000460203180800282C8316031351088312FC
:10387000D600561C3D2C85153E2C8511D61C422C9D
:103880000516432C0512561D472C85160800851277
:103890000800F401F5010310F30CF20C031C572C83
:1038A0007008F40771080318710AF5070310F00D8A
:1038B000F10D72087304031900344B2C83120313A7
:1038C00087010510831652088312D6005618071474
:1038D000D618871456190514D6198715561A0716BF
:1038E00085148514851008000A168A1126250A16E3
:1038F0008A1570088316B6007108B7007208B80000
:103900007308B9002408173E840083173608800026
:103910008312080083120313BE001F3E8400831726
:10392000023080003E08173E840083170C30800070
:103930003E08153E840083178001840A0830800009
:103940000800831203134C08F0004D08F1004E08E4
:10395000F2004F08F300CF1F0800F009F109F20947
:10396000F309F00A0319F10A0319F20A0319F30A19
:103970000800831203179515A215AF159030831612
:1039800003132406031DC82C831203179511D12C91
:10399000B030240683120317031DD02CA211D12CA2
:1039A000AF11831603132017831208008312031329
:1039B000A20126082707A000A007250DA100230EBD
:1039C0002307A0072708A107A00DA10D230E260796
:1039D000A007250E03180138A107270EA002031C1B
:1039E000A1030310A00DA10D03182214250E240716
:1039F000A007250803182503A1020313831208005A
:103A00000A168A1126250A168A1570088316B6002A
:103A10007108B7007208B8007308B9003804031DB4
:103A2000352D0A30F200F3013608F0003708F100B6
:103A30000A128A11D0260A168A157408B60075086B
:103A4000B70009303702C530031936020318352D87
:103A5000370836040319352D2408153E84008317D2
:103A600036088000840A3708800083120800831219
:103A70000313210E0F39DC3EA700A707983EA300D1
:103A8000903EA40021080F39A307A307A407DF3E37
:103A9000A600A607A607200E0F39A607A407A60DA5
:103AA000A40DA409A40D20080F39A407A70D1030F8
:103AB000A500221C632D0430A402A6070530A3072D
:103AC000A7070630A5070A30A407A603031C642D28
:103AD000A607A303031C682DA307A703031C6C2DD3
:103AE000A707A503031C702D03138312080083127C
:103AF00003138701051003179519812D03138714EC
:103B00000317A219862D031387150317AF198A2DE2
:103B10000313871603130610F4300A168A150C24B3
:103B20000614871087118712F4300A168A150C24A0
:103B30000A168A1507100510071203179519A32DE9
:103B4000031307140317A219A82D03130514031751
:103B5000AF19AC2D0313071603130610F4300A1621
:103B60008A150C240A168A15061407100510071268
:103B7000080083120313C3001F3E84008317023022
:103B800080004108C7004208C8004708A000480854
:103B9000A100A2010A168A1537250A168A152508DA
:103BA000CD002708CC002308CB002608CA00240833
:103BB000C9000430C6004608493E840083138008CB
:103BC000031DE42DC60BDB2DC50145084602031C71
:103BD00008004508493E840083130008C4004508D6
:103BE0004307193E8400831718308A0044084E208A
:103BF0000A168A158000C50AE52D83120313C10039
:103C00000A168A118E250A168A157008C2007108D4
:103C1000C3007208C4007308C5008316A01C132ECD
:103C200083124108162E83124108043E8400831734
:103C30000008F000840A0008F100840A0008F2007D
:103C4000840A0008F3007008C2077108031C2D2EB7
:103C5000710A0319F20A0319F30AC3077208031C55
:103C6000342E720A0319F30AC40773080318730A7F
:103C7000C5074108083E8400831742088000840A73
:103C800043088000840A44088000840A45088000B4
:103C90008316A01452148312080083160317EF082A
:103CA0000313031DAB2E4B088312A00083164C0890
:103CB0008312A10083164D088312A2000A168A15EA
:103CC000372518308A0024084E20C10018308A0099
:103CD00026084E20C20018308A0023084E20C30058
:103CE00018308A0027084E20C40018308A002508A2
:103CF0004E200A168A15C500C601A508031D8D2E83
:103D0000C501A708031D8D2EC401A308031D8D2E18
:103D1000C301A608031D8D2EC20141088316031797
:103D2000E90083120313420883160317EA00831283
:103D30000313430883160317EB008312031344088D
:103D400083160317EC008312031345088316031729
:103D5000ED00EE0103138312080083120313BD006C
:103D60008316A01CB72E83123D08083EBA2E83127C
:103D70003D08043E840083170008F000840A000810
:103D8000F100840A0008F200840A0008F3007008B9
:103D9000BE007108BF007208C0007308C1003D0872
:103DA000840083170008F000840A0008F100840AE8
:103DB0000008F200840A0008F3007008BE077108CA
:103DC000031CE72E710A0319F20A0319F30ABF074D
:103DD0007208031CEE2E720A0319F30AC007730857
:103DE0000318730AC107410DC10CC00CBF0CBE0CF7
:103DF0008316A01C0C2F83123D08083E84008317F5
:103E00003E088000840A3F088000840A4008800041
:103E1000840A41088000080083123D08043E8400A3
:103E200083173E088000840A3F088000840A400807
:103E30008000840A41088000080083120317170BD2
:103E40003A2F973018020318262F980A10300A12BA
:103E50008A15E12190300A128A157C2090300A16CA
:103E60008A11B7260A168A1503171208960002301F
:103E700097001512240B552F973025020318412F58
:103E8000A50A1D300A128A15E121B0300A128A15DE
:103E90007C20B0300A168A11B7260A168A15031735
:103EA0001F08A3000230A4002212310B772F973095
:103EB000320203185C2FB20A2A300A128A15E12155
:103EC000D0300A128A157C200A168A158316A01D86
:103ED000201A702FD0300A168A11B7260A168A15B2
:103EE000831203172C08B0000230B1002F121708FC
:103EF000023A03197D2F151E8C2F2408023A03194C
:103F0000832F221E8C2F3108023A0319892F2F1E6E
:103F10008C2F9701A401B10103130800831203132E
:103F2000CF004B08F4004C08F5004D08F6004E0891
:103F3000F7004F08153E840083170008F000840A3C
:103F40000008F100F201F3010A128A11B7270A16DC
:103F50008A157008D0007108D1007208D200730869
:103F6000D3003230D400D31FB72FD409D40A540859
:103F7000D00701300318D1070318D2070318D3075D
:103F80006430F400F501F601F7015030840083132A
:103F90000A128A1107270A168A1583160313201C92
:103FA000F52F3230F400F501F601F701831250309D
:103FB000840083130A128A11E52719308312031330
:103FC000D00701300318D1070318D2070318D3070D
:103FD0007F30F400F501F601F701503084008313BF
:103FE0000A128A1107270A168A158312031350082A
:103FF000F0005108F1005208F2005308F3000800E5
:02400E0076FF3B
:1042000000000000000000000000000000000000AE
:10421000000000000000000000000000000000009E
:10422000000000000000000000000000000000008E
:10423000000000000000000000000000000000007E
:10424000000000000000000000000000000000006E
:10425000000000000000000000000000000000005E
:10426000000000000000000000000000000000004E
:10427000000000000000000000000000000000003E
:10428000000000000000000000000000000000002E
:10429000000000000000000000000000000000001E
:1042A000000000000000000000000000000000000E
:1042B00000000000000000000000000000000000FE
:1042C00000000000000000000000000000000000EE
:1042D00000000000000000000000000000000000DE
:1042E00000000000000000000000000000000000CE
:1042F00000000000000000000000000000000000BE
:1043000000000000000000000000000000000000AD
:10431000000000000000000000000000000000009D
:10432000000000000000000000000000000000008D
:10433000000000000000000000000000000000007D
:10434000000000000000000000000000000000006D
:10435000000000000000000000000000000000005D
:10436000000000000000000000000000000000004D
:10437000000000000000000000000000000000003D
:10438000000000000000000000000000000000002D
:10439000000000000000000000000000000000001D
:1043A000000000000000000000000000000000000D
:1043B00000000000000000000000000000000000FD
:1043C00000000000000000000000000000000000ED
:1043D00000000000000000000000000000000000DD
:1043E00000000000000000000000000000000000CD
:1043F00000000000000000000000000000000000BD
:00000001FF
